:10000000C7FFA986DE9C0000E30100000003250075
:100010000127020E3C03000000000000400000C366
:100020004700000100030D00FFFC0000000000532A
:10003000000306090C0F1215181B1E21262B302059
:10004000000000000000000017050000000000E0B4
:1000500011060000000000C03509000000000090FB
:10006000000000000000009895000000000000A0C3
:1000700016010000000000A885010000000000B08B
:10008000F2010000000000B85D020000000000C0A6
:10009000C0020000000000C81B030000000000D0E8
:1000A00074030000000000D8C9030000000000E055
:1000B0001E040000000000E863040000000000F0DF
:1000C0009E040000000000F8D70400000000009526
:1000D0000000000000000001010101010101010117
:1000E0000101010101010101010101010101010100
:1000F00001010101010101010101010101010101F0
:1001000001010101010101010101010101010101DF
:1001100001010101010101010101010101010101CF
:101DD00001010101010101000000000000000000FC
:101DE00000000000000000000000000000000000F3
:101DF00000000000000000000000000000000000E3
:101E000000000000000000000000000000000000D2
:101E100000000000000000000000000000000000C2
:1023D00000000000000000020202020202020202EB
:1023E00002020202020202020202020202020202CD
:1023F00002020202020202020202020202020202BD
:1024000002020202020202020202020202020202AC
:10241000020202020202020202020202020202029C
:1040D00002020202020202000000000000000000D2
:1040E00000000000000000000000000000000000D0
:1040F00000000000000000000000000000000000C0
:1041000000000000000000000000000000000000AF
:10411000000000000000000000000000000000009F
:104CD00000000000000000010101010101010101CB
:104CE00001010101010101010101010101010101B4
:104CF00001010101010101010101010101010101A4
:104D00000101010101010101010101010101010193
:104D10000101010101010101010101010101010183
:1069D00001010101010101000000000000000000B0
:1069E00000000000000000000000000000000000A7
:1069F0000000000000000000000000000000000097
:106A00000000000000000000000000000000000086
:106A10000000000000000000000000000000000076
:106FD000000000000000000202020202020202029F
:106FE0000202020202020202020202020202020281
:106FF0000202020202020202020202020202020271
:107000000202020202020202020202020202020260
:107010000202020202020202020202020202020250
:108CD0000202020202020200000000000000000086
:108CE0000000000000000000000000000000000084
:108CF0000000000000000000000000000000000074
:108D00000000000000000000000000000000000063
:108D10000000000000000000000000000000000053
:1095D0000000000000000081000000000000000109
:1095E000010101010101010101010101010101016B
:1095F000010101010101010101010101010101015B
:10960000010101010101010101010101010101014A
:10961000010101010101010101010101010101013A
:10AED0000101010101010101010101010101010063
:10AEE0000000000000000000000000000000000062
:10AEF0000000000000000000000000000000000052
:10AF00000000000000000000000000000000000041
:10AF10000000000000000000000000000000000031
:10B4D000000000000000000000000000000000026A
:10B4E000020202020202020202020202020202023C
:10B4F000020202020202020202020202020202022C
:10B50000020202020202020202020202020202021B
:10B51000020202020202020202020202020202020B
:10CDD0000202020202020202020202020202020035
:10CDE0000000000000000000000000000000000043
:10CDF0000000000000000000000000000000000033
:10CE00000000000000000000000000000000000022
:10CE10000000000000000000000000000000000012
:10D7D0000000000000000000000000000000000148
:10D7E0000101010101010101010101010101010129
:10D7F0000101010101010101010101010101010119
:10D800000101010101010101010101010101010108
:10D8100001010101010101010101010101010101F8
